:108957009009FB7427F0A37410F09009FB74FFF5DE
:0F896700F0124DFEFED3E5F09400EE940050EBBD
:108976007D017F0412852C128D50128FEF128FD934
:0F898600128EDA124FDA128E1C128F4802909D59
:10852C00AE8475840F758A83E4F59775840FF5898D
:10853C00F58475B73075840F4389018D8D758F0166
:10854C008F8EFDFC0DBD00010CE4B505F7ECB401FC
:10855C00F3438902E58920E4120DEDAA0470010CA5
:10856C0014D39400EA6480948140E9759702AF06B5
:02857C008F84EA
:01857E0022DA
:108D5000AF8475840F75E10343E20443E3C075A457
:108D60000F7580F075A51775AD17E4F5A675A7F01A
:028D70008F84EE
:018D720022DE
:108FD900AF84E4F58475D48475840175D484F584EB
:058FE90075D1038F8427
:018FEE002260
:108FEF00AF84E4F584759D0443F808759A40D2F870
:028FFF008F845D
:01900100224C
:108E1C00AF8475840175C90875CA3C75CB5D75CA7C
:0F8E2C000175CB7075CD6E75CCACE4F5C88F8435
:018E3B002214
:108F4800AF84758402E4F5C975CA1975CBFF75CD70
:088F5800FF75CC19F5C88F84E8
:018F600022EE
:104FDA00900A0FE584F0E4F584F5BA75BC9875E893
:104FEA00C0758402F5BA75BC9043BC0175E8C0125D
:084FFA008BFF900A0FE0F58423
:01500200228B
:0A909D0043E701D2A8D28AD2AF2225
:0890B10033302E312020200095
:06839F00C10E4106A00022
:108B9700AE8475840F75A40F7580F075A7F0E4FD9A
:108BA700FC0DBD00010CBC4EF8BD20F5E58030E69C
:108BB70004E4FF800CE5B0540F70047F018002E4E9
:038BC700FF8E849A
:018BCA002288
:1050390075FFDE75FFADE4F5E6F5E79006A330945C
:10504900057444F080037445F01289579006A3E073
:10505900FF12906243F602129013E49005AEF090AD
:10506900069A7407F0E490069EF09006A2F0900468
:10507900BBF09005A8124F2500000000E490069BA4
:10508900F004A3F0E49006A6F0128E7C128B2C900B
:10509900069DE0FF129024129054128A821290EE1B
:1050A900127DB312906FE49005ACF0A3F075840102
:1050B90043C804F5849006A5F09005AD04F0758405
:1050C9000F7B017A097922128C8DEF70030253014B
:1050D900900924E0124F6251590451A605511B143D
:1050E90050FF16510E1751201A51421B514D1D5197
:1050F900531E000052019006A274FFF09005AD7492
:1051090001F0025201E49006A2F09005AD04F0020C
:105119005201D20E0252017B017A09792290093299
:10512900EBF0A3EAF0A3E9F0124CE5FE9006A3E048
:10513900FF6E600302520180059006A3E0FF128D05
:10514900FB0252011290C80252011290F40252015C
:105159007B017A097922900935EBF0A3EAF0A3E9FA
:10516900F0900003124CFEFF9006A3E06F6003026B
:1051790052019006A2E06078900935EBF0A3EAF0BD
:10518900A3E9F0900005124CFEFF900006124CFEB8
:10519900FD900004124CFEFB12800180537B017AC2
:1051A900097922900935EBF0A3EAF0A3E9F0900020
:1051B90003124CFEFF9006A3E06F703C9006A2E03C
:1051C900602E900935EBF0A3EAF0A3E9F090000511
:1051D900124CFEFF900006124CFEFD900004124C8A
:1051E900FEFB127F4B128B2C9005AC7401F0A3F0DF
:1051F9009006A3E0FF128E9C9006A2E07003025075
:10520900CA900924E014603524FA605D1470030221
:1052190052C4240660030250CA1290027B017A0923
:105229007922900932EBF0A3EAF0A3E9F0900003A8
:10523900124CFE9006A6F01290FA0252FB1290024E
:105249007B017A097922900932EBF0A3EAF0A3E90C
:10525900F0900003124CFE9006A6F0128B2C9005DC
:10526900AC7401F0A3F00252FB1290027B017A099F
:105279007922900938EBF0A3EAF0A3E9F090000352
:10528900124CFEFF900004124CFEFD900005124CDA
:10529900FEFBC003900938E0FBA3E0FAA3E0F99014
:1052A9000006124CFE90094AF0D003127E80128B40
:1052B9002C9005AC7401F0A3F080371290027B01A9
:1052C9007A097922900938EBF0A3EAF0A3E9F09082
:1052D9000003124CFEFF900004124CFEFD900005E5
:1052E900124CFEFB12734E128B2C9005AC7401F01C
:1052F900A3F012907C0250CA128EF7EF7003025885
:105309005912883DEFB41400400302585090531DC0
:10531900F828287302535902538C0253AB02539550
:105329000253BE0253DA02555302556D02558702E4
:1053390055F70256660256D50254760254E50257CD
:10534900430257B202582802583002537502584E88
:10535900300E099006A2E0F4F0025470E49006A61B
:10536900F01290FAE49006A5F0025470200E0302A0
:1053790058509006A3E0FF7BFF7A9079B11284CC54
:1053890002585090069EE0F4F0025470900699E09D
:1053990004F0A3E0FF900699E0D39F4031E4F002C6
:1053A900581E900698E0F4F0E490069BF09005AD45
:1053B90004F00258509005AEE004F0E0FFB4030495
:1053C900E4F0800AEFB4FF069005AE7402F00258CB
:1053D9001E900699E0FF75F01DA424B3F582E4340C
:1053E90005F583C083C0829005AEE0FED082D083EC
:1053F90075F009124F56E004F0EF75F01DA424B3BF
:10540900F582E43405F58375F009EE124F56E0FF95
:10541900B40827900699E075F01DA424B3F582E439
:105429003405F583C083C0829005AEE0D082D08375
:1054390075F009124F56E4F0802AEFB4FF26900662
:1054490099E075F01DA424B3F582E43405F583C011
:1054590083C0829005AEE0D082D08375F009124FE7
:10546900567407F01250309005AD025849900699CC
:10547900E0FF75F01DA424AFF582E43405F583C07F
:1054890083C0829005AEE0FED082D08375F0091208
:105499004F56E004F0EF75F01DA424AFF582E43413
:1054A90005F58375F009EE124F56E0D39455402661
:1054B900900699E075F01DA424AFF582E43405F552
:1054C90083C083C0829005AEE0D082D08375F00995
:1054D900124F567455F012503002581E900699E03A
:1054E900FF75F01DA424AFF582E43405F583C0836C
:1054F900C0829005AEE0FED082D08375F009124FCC
:1055090056E014F0EF75F01DA424AFF582E43405DC
:10551900F58375F009EE124F56E0D3945540259066
:105529000699E075F01DA424AFF582E43405F583EE
:10553900C083C0829005AEE0D082D08375F0091295
:105549004F56E4F012503002581E900879A3E0FA41
:10555900A3E0F5828A837F01124F8C1250309005A7
:10556900AC025849900879A3E0FAA3E0F5828A834E
:105579007FFF124F8C1250309005AC0258499006AB
:1055890099E0FF75F01DA424B0F582E43405F58394
:10559900C083C0829005AEE0FED082D08375F00949
:1055A900124F56E02402F0EF75F01DA424B0F582E5
:1055B900E43405F58375F009EE124F56E0D3946390
:1055C9004026900699E075F01DA424B0F582E434D4
:1055D90005F583C083C0829005AEE0D082D0837583
:1055E900F009124F567463F012503002581E90069B
:1055F90099E0FF75F01DA424B0F582E43405F58324
:10560900C083C0829005AEE0FED082D08375F009D8
:10561900124F56E024FEF0EF75F01DA424B0F58278
:10562900E43405F58375F009EE124F56E0D394631F
:105639004025900699E075F01DA424B0F582E43464
:1056490005F583C083C0829005AEE0D082D0837512
:10565900F009124F56E4F012503002581E90069984
:10566900E0FF75F01DA424B1F582E43405F583C08B
:1056790083C0829005AEE0FED082D08375F0091216
:105689004F56E004F0EF75F01DA424B1F582E4341F
:1056990005F58375F009EE124F56E0D39463402661
:1056A900900699E075F01DA424B1F582E43405F55E
:1056B90083C083C0829005AEE0D082D08375F009A3
:1056C900124F567463F012503002581E900699E03A
:1056D900FF75F01DA424B1F582E43405F583C08378
:1056E900C0829005AEE0FED082D08375F009124FDA
:1056F90056E014F0EF75F01DA424B1F582E43405E9
:10570900F58375F009EE124F56E0D3946340259066
:105719000699E075F01DA424B1F582E43405F583FA
:10572900C083C0829005AEE0D082D08375F00912A3
:105739004F56E4F012503002581E900699E0FF755A
:10574900F01DA424B2F582E43405F583C083C08238
:105759009005AEE0FED082D08375F009124F56E075
:105769002402F0EF75F01DA424B2F582E43405F5A6
:105779008375F009EE124F56E0D3946340269006E4
:1057890099E075F01DA424B2F582E43405F583C0CF
:1057990083C0829005AEE0D082D08375F009124FA4
:1057A900567463F0125030806C900699E0FF75F0E2
:1057B9001DA424B2F582E43405F583C083C0829028
:1057C90005AEE0FED082D08375F009124F56E02471
:1057D900FEF0EF75F01DA424B2F582E43405F583DB
:1057E90075F009EE124F56E0D3946340259006995F
:1057F900E075F01DA424B2F582E43405F583C08375
:10580900C0829005AEE0D082D08375F009124F5660
:10581900E4F01250309005AC7401F0A3F080281226
:105829008E3C9005AC80199006A0E0F4F07005124A
:10583900501B800990D000E49390069DF09005AC30
:105849007401F0800280FE128EF7EF600302530AA2
:105859009005ADE06008125D7CE49005ADF090051F
:10586900ACE070030250C712906FE49005ACF002EF
:0258790050C716
:10891300AB84A2AF920FE4FCFDED9009D9124F197D
:108923009009DBE0FEA3E07816A60608F6E4F584DA
:10893300C2AF43B701438F02438F0118E6FE08E637
:10894300F5828E83E4F053B7FEF58FA20F92AFAF9B
:03895300038F840B
:0189560022FE
:02857F00AB054A
:10858100AA84A2AF9210E4FCFDED9009DD124F190F
:10859100EBFF3395E0FEEFF44E60299009DFE0FE3A
:1085A100A3E07818A60608F6E4F584C2AF43B70144
:1085B100758F0118E6FC08E6F5828C83EBF053B762
:0C85C100FEE4F58FA21092AFAF028F8491
:0185CD00228B
:10846B009009C1EEF0A3EFF0A3ECF0A3EDF0A3EABB
:10847B00F0A3EBF09009C5E07002A3E06042900915
:10848B00C1E0FEA3E0FFA3E0FCA3E0F5828C83E058
:10849B00FD12857F9009C6E024FFF09009C5E034FA
:1084AB00FFF09009C4E004F070069009C3E004F0FB
:1084BB009009C2E004F070BC9009C1E004F080B4F4
:0184CB00228E
:0890B900E4900000F0A3F02296
:108CE000900000E0FEA3E0FF128913900000E0FE78
:108CF000A3E0FF7C007D027B007A0412846BE49089
:068D00000000F0A3F022C8
:0A812C00A9059009C7EEF0A3EFF0DB
:10813600EE54FCFE900000E0FCA3E0FD7002EE6C45
:108146006057ED4C6003128CE09009C7E0FEEE54D8
:10815600FCFE7F00900000F0A3EFF09009C9EEF05E
:10816600A3EFF0A37400F0A37402F07E049009C993
:10817600E475F001124DFE85F082F583E493FD90DF
:1081860009CBE475F001124DFE85F082F583EDF022
:10819600EF1F70011EEF4E70D49009C7E0FCA3E0FC
:1081A600FDEC5403FC74022DF58274003CF583E962
:0181B600F0D8
:0181B70022A5
:108888009009B3EEF0A3EFF0A3EBF0A3EAF0A3E9AD
:10889800F09009B874FFF5F0124DFE45F06026908F
:1088A80009B3E475F001124DFEAFF0FE9009B5E092
:1088B800FBA3E475F001124DFEA9F0FA124CE5FD98
:0688C80012812C80CC227D
:1083A500420873000042081E00004208190000C17F
:0583B5000BC10AC10923
:0A90A700C20AC20BE490081DF0227B
:108D7300E4900873F0A3F090081EF0A3F0A3F09022
:108D83000819F0A3F0900814F0A37440F0E49008DD
:038D93001CF022AF
:0690D6001290A7028D7349
:108F6100E4F5848FC343C30175C04475CF8EC2C37A
:098F710043E60290081B04F02203
:10900200E4F58420C7FDC2C21290D6E490081BF09A
:01901200223B
:0B907C00E4F584D2C290081B04F0222F
:0D906200AE07128F61900818EFF00290D653
:108D0600E49009FDF0A3F0300A02FF22200BFDD209
:108D16000A900816E4F0A37410F0900861EFF0E4EE
:048D2600A3F07F0136
:018D2A002226
:108BCB00300A0A900816E07002A3E070037F0022BF
:108BDB00900817E024FFF0900816E034FFF090089F
:108BEB0062E0FE04F074632EF582E43408F583EF43
:048BFB00F07F0122E4
:0B908700300A07C20AD20B12904522EB
:0E904500AF84E4F58420C7FDC2C4D2C58F8479
:0190530022FA
:1082B7009009BBEBF0A3EAF0A3E9F090081BE0708C
:1082C70002FF229009BEE0FE6005D3941040037FB1
:0882D7000022128D06EF604E3B
:1082DF00E49009C0F09009BEE0FF9009C0E0FEC332
:1082EF009F50249009BBE0FBA3E0FAA3E0F98E8234
:1082FF00758300124CFEFF128BCBEF7002FF2290A2
:10830F0009C0E004F080CEE490081DF01290879031
:0E831F0009BFE07003200BFD90081DE0FF2257
:03832D007FFF22AD
:0E7AB9009009E1EBF0A3EAF0A3E9F0A3EDF0F1
:107AC700E4FFD3900874E09400900873E064809416
:107AD7008050012253E6FD900819E0FEA3E0242020
:107AE700F58274083EF583E0FF900819E475F0010C
:107AF700124DE8FCE5F064404C7006900819F0A3BD
:107B0700F0900815E004F07006900814E004F0E423
:107B1700FE9009E4E0FDEEC39D5054EEC39F504F25
:107B2700900819E0FCA3E02420F58274083CF58353
:107B3700E0FD9009E1E0FBA3E0FAA3E0F98E82758E
:107B47008300ED124D5F900819E475F001124DE8BE
:107B5700FCE5F064404C7006900819F0A3F090081B
:107B670015E004F07006900814E004F00E80A2EE11
:107B7700C39F5029900819E475F001124DE8FCE500
:107B8700F064404C7006900819F0A3F0900815E0D7
:107B970004F07006900814E004F00E80D290087488
:107BA700E024FFF0900873E034FFF043E602900909
:0C7BB700E4E0FEEFC39E50028002AF0627
:017BC300229F
:108F9300D3900874E09400900873E0648094804058
:088FA300047F0180027F00221F
:0350180002795BBF
:10795B00C0E0C0F0C083C082C0D075D000C000C0F2
:03796B0006C0074C
:10796E00C211AFC1EF124F6279A40879A41079B495
:10797E001879B92079C62879F33079FE387A0660FD
:10798E007A01687A06707A01787A0E807A0E907A89
:10799E0085A000007A93900861E0F5C2C2C59008F8
:1079AE0060E4F0027A95900862802890081D74FDBC
:1079BE00F0D2C4D2C5027A95900862E0FF900860BA
:1079CE00E0C39F5014E0FF04F074632FF582E4349B
:1079DE0008F583E0F5C2027A95D2C490081DE4F052
:1079EE00C20B027A95D2C590081D74FEF0027A95EC
:1079FE00027A8AD209027A95900813E4F0027A95F7
:107A0E00900813E07020E5C2F0E0FFC3900815E087
:107A1E009F7480F8900814E06480985003128D7360
:107A2E00900813E004F0900815E024FFF09008147D
:107A3E00E034FFF090081EE0FEA3E02420F58274EF
:107A4E00083EF583E5C2F090081EE475F001124D74
:107A5E00E8FEE5F064404E700690081EF0A3F0902C
:107A6E000813E014F07020900874E004F070189081
:107A7E000873E004F0801030090DC209900860E42C
:107A8E00F0D2C58002D21130110EC2C6D2C6C2C506
:0A7A9E00C2C4D2C2C211C20BC2C39F
:107AA800D007D006D000D0D0D082D083D0F0D0E09C
:017AB800329B
:0590DC00A2C7E433FF10
:0190E100226C
:0690E200C2C253E6FD22AC
:10768700900991E0FFA3E0FCA3E0FDA3E0FBA3E0EA
:10769700FAA3E0F9900941E512F0E513A3F0900988
:0676A70099E0900943F098
:1076AD0090093BEFF0A3ECF0A3EDF0A3EBF0A3EA10
:0476BD00F0A3E9F05D
:1076C1009009447403F0A374E8F0A3E584F0E4F5B1
:1076D1008420C7FDC2C4D2C2D2C5E4FF900A11F012
:1076E10030C3FDAEC1EE24F8602324F8601F24F8F6
:1076F100602F24F8603624F8603A24F8700302778A
:107701009924F870030277A124380277A9EF700C4D
:1077110090093BE025E044A0F5C27F03C2C5027792
:10772100AF90093CE0F5C27F050277AF900A117472
:1077310003F0807AEFB4050B90093CA3E0F5C27F1A
:1077410006806BEF6406703E900943E090093E703D
:107751000FE0FBA3E475F001124DFEA9F0FA8008D9
:10776100E0FBA3E0FAA3E0F9124CE5F5C29009426F
:10777100E024FFF0900941E034FFF0E07002A3E063
:10778100702C7F078028EFB40706D2C47F09801EC2
:10779100900A117405F08016900A117404F0800E9D
:1077A100900A117406F08006900A117401F0EFB48A
:1077B1000904C2C38036900A11E0B4031C90094445
:1077C10074FFF5F0124DE845F0600ED2C4D2C5D277
:1077D100C2C2C3E4900A11F0FF900A11E06008C22E
:1077E100C5D2C4C2C38005C2C30276E120C7FD90E1
:0577F1000946E0F584EB
:0177F6002270
:1077F700900953EFF0A3ECF0A3EDF0A3EBF0A3EAAD
:04780700F0A3E9F011
:10780B0090095B7403F0A374E8F0A3E584F0E4F54E
:10781B008420C7FDD2C2C2C4D2C5E4FF900A11F0C6
:10782B0030C3FDAEC1EE124F62785900785C087818
:10783B005C10788718789220789A2878B53078BDC4
:10784B003878C54078D550790758000078590279B7
:10785B000DC2C5EF700F900953E025E044A0F5C2AF
:10786B007F03027913EF64016003027913900953CC
:10787B00E025E044A1F5C27F04027913900954E09E
:10788B00F5C27F05027913900A117403F08079EF2A
:10789B00B4050B900954A3E0F5C27F06806AEFB4E0
:1078AB000606D2C57F0180608018900A117404F01F
:1078BB008056900A117406F0804EEFB404047F02D8
:1078CB008046900A117405F0803E900956E0FBA3A8
:1078DB00E475F001124DFEA9F0FAE5C2124D4D9080
:1078EB00095AE024FFF0900959E034FFF0E07002F0
:1078FB00A3E07004C2C280107F02800CD2C47F0947
:10790B008006900A117401F0EFB40904C2C38036EB
:10791B00900A11E0B4031C90095B74FFF5F0124D53
:10792B00E845F0600ED2C4D2C5D2C2C2C3E4900AFD
:10793B0011F0FF900A11E06008C2C5D2C4C2C38027
:0F794B0005C2C302782B20C7FD90095DE0F584CB
:01795A00220A
:107BC400900991EFF0900994EBF0A3EAF0A3E9F0A7
:087BD400900992ECF0A3EDF022
:107BDC00751400543FF515543F605CC37440951503
:107BEC00FFE49514FE900997E0FCA3E0FDC39FEC25
:107BFC009E50068C128D1380048E128F1312768772
:107C0C00900A11E060037F0222900993E02513F0A3
:107C1C00900992E03512F0900999E0700B9009955B
:107C2C00E5128513F0124DE8C3900998E09513F016
:107C3C00900997E09512F0900997E0F512A3E0F502
:107C4C0013D3E5139400E51294004070E5139440AF
:107C5C00E51294005013127687900A11E060037FAE
:107C6C000222E4F512F51380D8900991E0FFA3E00D
:107C7C00FCA3E0FDA3E0FBA3E0FAA3E0F99009412B
:107C8C00E4F074401276A3900A11E060037F0222A4
:107C9C0074C02513F51374FF3512F512900993E097
:107CAC002440F0900992E03400F0900999E0709132
:0E7CBC0090099575F040124DE8027C4D7F0056
:017CCA002297
:108FAB00900959E4F0A304F01277F7900A11E060EE
:078FBB00037F01227F002269
:108F1400900A10EBF07B017A0A7910900997E4F03B
:0A8F2400A304F0E4A3F0127BC422C2
:108D9600C0079009A9E0FFA3E0900959CFF0A3EF1F
:108DA600F0D0071277F7900A11E060037F01227F67
:028DB600002299
:108F2E00C0079009B1E0FFA3E0900997CFF0A3EF3F
:0A8F3E00F0E4A3F0D007127BC42278
:0E88CE009009CDEBF0A3EAF0A3E9F0A3EDF0E2
:1088DC00E49009D2F09009CDE0FBA3E0FAA3E0F913
:1088EC00A3E09009BEF09009D1E09009BFF0E4FF3D
:1088FC001282B7EFB4FF0D9009D2E0FE04F0EEC384
:06890C00940340D17E003F
:018912002242
:0B8C8D009009F5EBF0A3EAF0A3E9F07A
:108C98007E007F007D10124F8E9009F5E0FBA3E067
:108CA800FAA3E0F97D10127AB9EF7002FF227F0172
:018CB8002299
:1084CC009009697422F0A3EFF0A37413F0124CE539
:1084DC0090096CF0900001124CFE90096DF0900028
:1084EC0002124CFE90096EF0900003124CFE9009A3
:1084FC006FF0900004124CFE900970F09000051281
:10850C004CFE900971F0900006124CFE900972F02E
:10851C007B017A097969E49009D1F07D0A0288CE51
:108DDA009009E57422F0A3EFF0A37403F0A374FFE3
:108DEA00F07B017A0979E5E49009D1F07D040288E3
:018DFA00CEAA
:108DFB009009E97422F0A3EFF0A3741CF0A374FFA5
:108E0B00F07B017A0979E9E49009D1F07D040288BD
:018E1B00CE88
:108E9C00E49009EDF0A3EFF0A3740AF0A3EFF07BDC
:0F8EAC00017A0979EDE49009D1F07D040288CEB6
:108EDA007F80900793E4F0A3DFFC7B017A07799304
:0C8EEA008B0A8A0B890C8A088909D2B413
:018EF6002259
:108EF700E50A850B83850C826401700AE5096582A2
:0D8F07007004E50865837002FF227F0122DF
:10883D00E50A850B83850C826401700AE509658262
:10884D007004E50865837003FF802FAB0A050CE506
:10885D000CAA0B7002050B14F9124CE5FF74019074
:10886D0008136B700AE50C65827004E50B65837067
:0A887D0009750A01750B07750C93CD
:0188870022CE
:035003000284071D
:10840700C0E0C083C082C0D075D000C004C005C022
:0384170006C00795
:10841A00AF8475840FE5B0540FFEE58054801313C2
:10842A0013541F4EFE0509E509AC0870020508142D
:10843A00F5828C83EEF0C3E5099413E508940840AD
:10844A0006750807750993C2B43086FDD2B48F84C5
:10845A00D007D006D005D004D0D0D082D083D0E0C7
:01846A0032DF
:1083BA004308CF4020104808D2401004014010045E
:1083CA00014808C780200802802008024808EA02FB
:1083DA00020202010101014808DA02020202010155
:1083EA0001014808F200020408060A0C0E4808E2D5
:0883FA0000020406010305075F
:105D7C00900A00E5E7F0129092900698E0FD60071B
:105D8C009008BFE04480F09008BFE0FF9005AEE0C3
:105D9C00FE24CFF582E43408F583E0FCEF4C900848
:105DAC00BFF0ED7003025E39900697E06025C3905A
:105DBC0004B8E09401501C9008EAE024BFF582E49A
:105DCC003408F583C083C082E0FF9008D2E0FDEF79
:105DDC004D80559004BAE090069B6023E024EAF5D0
:105DEC0082E43408F583E024BFF582E43408F583BB
:105DFC00C083C082E0FF9008D2E0FDEF4D8029E027
:105E0C00FF24EAF582E43408F583E024BFF582E44C
:105E1C003408F583C083C082E0FD74D22FF582E490
:105E2C003408F583E0FFED4FD082D083F0900699D3
:105E3C00E0FF24DAF582E43408F583E024BFF58230
:105E4C00E43408F583C083C082E0FD74C72FF5826B
:105E5C00E43408F583E0FFED4FD082D083F0900856
:105E6C00BFE0FF900699E0FD75F01DA424B3F58208
:105E7C00E43405F58375F009EE124F56E025E0FE8B
:105E8C00EF4E9008BFF09008C5E0FF90069EE054DE
:105E9C0040FEEF4E9008C5F0300E07E0FF9006A2D2
:105EAC0080089008C5E0FF9006A5E05480FEEF4EF8
:105EBC009008C5F0900698E0FF600790069BE0FE06
:105ECC008002AE05EE75F01DA424B3F582E4340512
:105EDC00F583E024E2F582E43408F583E0C433333F
:105EEC0054C09008C6F0E0FEEF600790069BE0FF00
:105EFC008005900699E0FFEF75F01DA424BCF58297
:105F0C00E43405F583E024E2F582E43408F583E01B
:105F1C0033333354F84E9008C6F0E0FF900698E007
:105F2C00600790069BE0FE8005900699E0FEEE75FA
:105F3C00F01DA424C5F582E43405F583E024E2F5D4
:105F4C0082E43408F583E04F9008C6F0900699E09F
:105F5C0075F01DA424B1F582E43405F583C083C02B
:105F6C00829005AEE0D082D08375F009124F56E0D6
:105F7C00FFC3945040089008C4740FF0802DEFC3F9
:105F8C00943C40089008C47427F0801FEFC39428F9
:105F9C0040089008C47433F08011EFC39414900837
:105FAC00C440057439F08003743CF0900699E07598
:105FBC00F01DA424B0F582E43405F583C083C082BF
:105FCC009005AEE0D082D08375F009124F56E0FDFB
:105FDC00C3945040099008C5E0440FF08054EDC3C1
:105FEC00943C40099008C5E04427F0804590069900
:105FFC00E075F01DA424B0F582E43405F583C0836C
:10600C00C0829005AEE0D082D08375F009124F5655
:10601C00E0FDC3942840099008C5E04433F0801299
:10602C00EDC394149008C5E040054439F080034456
:10603C003CF0900699E075F01DA424B2F582E4348E
:10604C0005F583C083C0829005AEE0D082D0837505
:10605C00F009124F56E0FDC3945040099008C2E07D
:10606C00440FF08054EDC3943C40099008C2E044C6
:10607C0027F08045900699E075F01DA424B2F582B6
:10608C00E43405F583C083C0829005AEE0D082D0A5
:10609C008375F009124F56E0FDC39428400990080F
:1060AC00C2E04433F08012EDC394149008C2E04077
:1060BC00054439F08003443CF0900699E075F01DDE
:1060CC00A424AFF582E43405F583C083C082900527
:1060DC00AEE0D082D08375F009124F56E0FDC39428
:1060EC0048400A9008C3E0443FF0026190EDC3942D
:1060FC003C400A9008C3E0449FF0026190900699DE
:10610C00E075F01DA424AFF582E43405F583C0835B
:10611C00C0829005AEE0D082D08375F009124F5644
:10612C00E0FDC3943040099008C3E044CFF08054A4
:10613C00EDC3942440099008C3E044E7F0804590F7
:10614C000699E075F01DA424AFF582E43405F583BF
:10615C00C083C0829005AEE0D082D08375F0091266
:10616C004F56E0FDC3941840099008C3E044F3F087
:10617C008012EDC3940C9008C3E0400544F9F08004
:10618C000344FCF053E7FEC291E4FFE4FE74BF2F1E
:10619C00F582E43408F583E0FDA806088002C313F9
:1061AC00D8FC139292E49009FFF09009FFE004F000
:1061BC00E0B414F6D290E49009FFF09009FFE004EB
:1061CC00F0E0B414F6C2900EEEB408C10FEFB408B0
:1061DC00BAD291E49009FFF09009FFE004F0E0B42A
:1061EC0014F6C291900698E0600790069BE0FF8041
:1061FC0005900699E0FFEF75F01DA424B3F582E439
:10620C003405F583E030E104D2928002C292900A08
:04621C0000E0F5E7C2
:01622000225B
:0A9092007F089008BFE4F0A3DFFCA4
:01909C0022B1
:10587B002E3031002E3032002E3033002E303400DB
:10588B002E3035002E3036002E3037002E303800BB
:10589B002E3039002E3130002E3132002E313400B3
:1058AB002E3136002E3138002E3230002E3235009C
:1058BB002E3330002E3335002E3430002E3435008D
:1058CB002E3530002E3630002E3730002E3830007B
:1058DB002E393000312E3000312E3200312E340073
:1058EB00312E3600312E3800322E3000322E35005C
:1058FB00332E3000332E3500342E3000342E35004D
:10590B00352E3000362E3000372E3000382E30003A
:10591B00392E300031302E00467265650053757399
:10592B007400456E626C0050756C730053746F702D
:10593B00004379636C002020333100202033330087
:10594B00202033350020203337002020333900202E
:10595B002034310020203434002020343600202025
:10596B0034390020203532002020353500202035F9
:10597B0038002020363200202036350020203639E2
:10598B000020203733002020373800202038320009
:10599B0020203837002020393300202039380020D0
:1059AB00313034002031313000203131370020319B
:1059BB003233002031333100203133390020313480
:1059CB003700203135360020313635002031373560
:1059DB000020313835002031393600203230380084
:1059EB002032323000203233330020323437002063
:1059FB003236320020323737002032393400203330
:105A0B003131002033333000203334390020333729
:105A1B00300020333932002034313500203434301B
:105A2B000020343636002034393400203532330030
:105A3B0020353534002035383700203632320020FF
:105A4B0036353900203639390020373430002037CD
:105A5B0038340020383331002038383000203933C7
:105A6B0032002039383800313035300031313130A7
:105A7B0000313137300031323430003133323000C5
:105A8B00313430300031343830003135373000317B
:105A9B003636300031373630003138363000313958
:105AAB003830003230393000323232300032333558
:105ABB00300032343930003236343000323739303E
:105ACB00003239363000333134300033333230006A
:105ADB00333532300033373330003339353000341F
:105AEB00313930002531733A253264202531733A30
:105AFB00253264202531733A257300610041006221
:105B0B00004200660046002531733A25326420437B
:105B1B006E74726C20566C746765006D004D0025B9
:105B2B0031733A2532642025347320543A2533736C
:105B3B0000436F6E747261737420253164202020D2
:105B4B00202020002020202020202020202020206A
:105B5B002020202000204142434445464748494AE3
:105B6B004B4C4D4E4F505152535455565758595A02
:105B7B006162636465666768696A6B6C6D6E6F7092
:105B8B007172737475767778797A30313233343544
:105B9B00363738397E21402324255E262A28292DA5
:105BAB002B3D7CFF587BFF587FFF5883FF5887FFA7
:105BBB00588BFF588FFF5893FF5897FF589BFF58F0
:105BCB009FFF58A3FF58A7FF58ABFF58AFFF58B321
:105BDB00FF58B7FF58BBFF58BFFF58C3FF58C7FF4D
:105BEB0058CBFF58CFFF58D3FF58D7FF58DBFF5880
:105BFB00DFFF58E3FF58E7FF58EBFF58EFFF58F371
:105C0B00FF58F7FF58FBFF58FFFF5903FF5907FFDA
:105C1B00590BFF590FFF5913FF5917FF591BFF5909
:105C2B001FFF5923FF5928FF592DFF5932FF5937B1
:105C3B00FF593CFF5941FF5946FF594BFF5950FF44
:105C4B005955FF595AFF595FFF5964FF5969FF595D
:105C5B006EFF5973FF5978FF597DFF5982FF5987A2
:105C6B00FF598CFF5991FF5996FF599BFF59A0FF84
:105C7B0059A5FF59AAFF59AFFF59B4FF59B9FF599D
:105C8B00BEFF59C3FF59C8FF59CDFF59D2FF59D792
:105C9B00FF59DCFF59E1FF59E6FF59EBFF59F0FFC4
:105CAB0059F5FF59FAFF59FFFF5A04FF5A09FF5ADA
:105CBB000EFF5A13FF5A18FF5A1DFF5A22FF5A277D
:105CCB00FF5A2CFF5A31FF5A36FF5A3BFF5A40FFFF
:105CDB005A45FF5A4AFF5A4FFF5A54FF5A59FF5A17
:105CEB005EFF5A63FF5A68FF5A6DFF5A72FF5A776D
:105CFB00FF5A7CFF5A81FF5A86FF5A8BFF5A90FF3F
:105D0B005A95FF5A9AFF5A9FFF5AA4FF5AA9FF5A56
:105D1B00AEFF5AB3FF5AB8FF5ABDFF5AC2FF5AC75C
:105D2B00FF5ACCFF5AD1FF5AD6FF5ADBFF5AE0FF7E
:105D3B005AE5FF5AEA0105FF750E010EFF81B80007
:105D4B0000FF861D0005FF866B000AFF86B9010068
:105D5B00FF87070105FF750E0000FF861D0005FF7D
:105D6B00866B000AFF86B90100FF87070009FF8CCD
:015D7B002FF8
:0E905400E490089CF090089BF090089AF0229F
:0690E800E4900878F0227C
:10809700900A01EEF0A3EFF0AF051DEF7003028128
:1080A7002B900A01E0FEA3E0F5828E83A3A3E4935D
:1080B700FB740193FA740293F9900878E0FF75F066
:1080C70005A4247EF582E43408F583EBF0A3EAF0F7
:1080D700A3E9F0900A01E0FAA3E0FBF5828A83E4C2
:1080E70093FEEF75F005A4247CF582E43408F5834C
:1080F700EEF08B828A83740193FF900878E075F025
:1081070005A4247DF582E43408F583EFF090087820
:10811700E004F0900A02E02405F0900A01E0340040
:05812700F002809F2220
:10823B00900878E0FF6074900875E0FBA3E0FAA368
:10824B00E0F9124CE5C39F4004E4124D4D900875C4
:10825B00E0FBA3E0FAA3E0F9124CE5FE75F005A4F0
:10826B00247CF582E43408F583E0FFEE75F005A479
:10827B00247DF582E43408F583E0FD128FC290086B
:10828B0075E0FBA3E0FAA3E0F9124CE575F005A449
:10829B00247EF582E43408F583E0F9A3E0FAA3E049
:0C82AB00900879C9F0A3EAF0A3E9F022E2
:108E3C00900875E0FBA3E0FAA3E0F97401124D2B46
:108E4C00124CE5FF900878E0B50704E4124D4D2272
:108C2F00D3EF64809480401190069DE004F0E0D370
:108C3F00940740137407F0800E90069DE014F0E047
:0F8C4F00D394074002E4F090069DE0FF029024CA
:10750E00900697E06003027623D3EF648094804068
:10751E006C900699E0FD75F01DA424CBF582E43441
:10752E0005F583E004F0ED75F01DA424CBF582E49F
:10753E003405F583E0FDD394054021900699E0755E
:10754E00F01DA424CBF582E43405F5837405F09088
:10755E0006977401F090069A7407F022ED640460A9
:10756E0075900699E075F01DA424CBF582E43405E0
:10757E00F583E06405600302768602764B900699E9
:10758E00E0FD75F01DA424CBF582E43405F583E00F
:10759E0014F0ED75F01DA424CBF582E43405F583CB
:1075AE00E0FDD394054014900699E075F01DA424D7
:1075BE00CBF582E43405F583E4F022ED6404601625
:1075CE00900699E075F01DA424CBF582E43405F500
:1075DE0083E0FDB405028065ED64036003027686E8
:1075EE0090069A7407F0900699E004FEEEC3940894
:1075FE004003027686EE75F01DA424CBF582E434AA
:10760E0005F583E0FD64046004EDB4050590069A6B
:10761E00EEF00E80D7D3EF64809480505BE490063A
:10762E0097F0900699E075F01DA424CBF582E43412
:10763E0005F583E0FF64046004EFB4050990069934
:10764E00E090069AF02290069A7407F0900699E060
:10765E0004FEEEC394085020EE75F01DA424CBF565
:10766E0082E43405F583E0FF64046004EFB405059D
:08767E0090069AEEF00E80DA8E
:0176860022E1
:1081B800D3EF64809480403E900699E0FF75F01DEF
:1081C800A424CAF582E43405F583E004F0EF75F0E1
:1081D8001DA424CAF582E43405F583E0C39429403C
:1081E80051900699E075F01DA424CAF582E434057F
:1081F800F5837429F022900699E0FF75F01DA424F8
:10820800CAF582E43405F583E014F0EF75F01DA497
:1082180024CAF582E43405F583E0C3942940139019
:108228000699E075F01DA424CAF582E43405F583A7
:03823800E4F0224D
:10861D00D3EF64809480900699E075F01D4020A4FE
:10862D0024B4F582E43405F583C083C0829005AE91
:10863D00E0D082D08375F009124F567401F022A458
:10864D0024B4F582E43405F583C083C0829005AE71
:0E865D00E0D082D08375F009124F56E4F0226F
:10866B00D3EF64809480900699E075F01D4020A4B0
:10867B0024B5F582E43405F583C083C0829005AE42
:10868B00E0D082D08375F009124F567401F022A40A
:10869B0024B5F582E43405F583C083C0829005AE22
:0E86AB00E0D082D08375F009124F56E4F02221
:1086B900D3EF64809480900699E075F01D4020A462
:1086C90024B6F582E43405F583C083C0829005AEF3
:1086D900E0D082D08375F009124F567401F022A4BC
:1086E90024B6F582E43405F583C083C0829005AED3
:0E86F900E0D082D08375F009124F56E4F022D3
:10870700D3EF64809480900699E075F01D4020A413
:1087170024B7F582E43405F583C083C0829005AEA3
:10872700E0D082D08375F009124F567401F022A46D
:1087370024B7F582E43405F583C083C0829005AE83
:0E874700E0D082D08375F009124F56E4F02284
:106DD9001290E89008FD74FFF0A3745AF0A374EFC1
:106DE900F0900699E075F01DA424B4F582E4340509
:106DF900F583C083C0829005AEE0D082D08375F060
:106E090009124F56E07BFF60067A5B790680047AA7
:106E19005B7908900900EBF0A3EAF0A3E9F090068A
:106E290099E0FF75F01DA424B0F582E43405F583DB
:106E3900C083C0829005AEE0FED082D08375F00990
:106E4900124F56E0FD900903E4F0A3EDF0EF75F061
:106E59001DA424B5F582E43405F58375F009EE1215
:106E69004F56E07BFF60067A5B790A80047A5B798A
:106E79000C900905EBF0A3EAF0A3E9F0900699E07C
:106E8900FF75F01DA424B1F582E43405F583C083B0
:106E9900C0829005AEE0FED082D08375F009124F12
:106EA90056E0FD900908E4F0A3EDF0EF75F01DA49C
:106EB90024B6F582E43405F58375F009EE124F56D0
:106EC900E07BFF60067A5B790E80047A5B7910902B
:106ED900090AEBF0A3EAF0A3E9F0900699E075F04E
:106EE9001DA424AFF582E43405F583C083C08290E4
:106EF90005AEE0D082D08375F009124F56E075F0E7
:106F090003A4243EF582E5F0345CF583E493F97437
:106F19000193FA74029390090DC9F0A3EAF0A3E969
:106F2900F07B017A08799D126AD9900697E070037F
:106F3900026FCB9008FD74FFF0A3745BF0A3741289
:106F4900F0900699E0FF75F01DA424B7F582E434AA
:106F590005F583C083C0829005AEE0FED082D08360
:106F690075F009124F56E07BFF60067A5B7926803F
:106F7900047A5B7928900900EBF0A3EAF0A3E9F021
:106F8900EF75F01DA424B2F582E43405F58375F09C
:106F990009EE124F56E0FF900903E4F0A3EFF07BEE
:106FA900017A0879AE126AD97E5D7F5E7D0512800D
:106FB900979008757401F0A37408F0A3749BF0020C
:106FC90070BC9008FD74FFF0A3745BF0A3742AF001
:106FD900900699E0FF75F01DA424B7F582E4340505
:106FE900F583C083C0829005AEE0FED082D0837560
:106FF900F009124F56E07BFF60067A5B7926800420
:107009007A5B7928900900EBF0A3EAF0A3E9F0EFA5
:1070190075F01DA424B2F582E43405F58375F009F1
:10702900EE124F56E0FD900903E4F0A3EDF0EF7581
:10703900F01DA424CBF582E43405F583E075F00353
:10704900A4242CF582E4345CF583E493F974019368
:10705900FA740293900905C9F0A3EAF0A3E9F09044
:107069000699E075F01DA424CAF582E43405F58378
:10707900E075F003A424AEF582E4345BF583E49370
:10708900F9740193FA740293900908C9F0A3EAF01C
:10709900A3E9F07B017A0879AE126AD97E5D7F4057
:1070A9007D061280979008757401F0A37408F0A307
:1070B900749AF09009D67401F0A37408F0A374AE21
:0D70C900F07B017A08799D128A4902823B12
:108330001290E89008FD74FFF0A3745BF0A3743C06
:10834000F090069DE0FF900900E4F0A3EFF07B01C0
:108350007A08799D126AD99008FD74FFF0A3745BC6
:10836000F0A3744FF07B017A0879AE126AD97E5D72
:108370007F777D011280979008757401F0A37408CF
:10838000F0A3749CF09009D67401F0A37408F0A3D4
:0F83900074AEF07B017A08799D128A4902823B14
:0D906F009006A0E06003028330126DD9224C
:1087550000010204081000000304180000000000D6
:108765001F000000000018040300000000100804AA
:1087750002010000040A0A11110000010102021C95
:1087850000001C020201010000101008080700008B
:0E8795000708081010000020406080A0C0FF00
:109013007F38128EBB7F06128EBB7D0EE4FF02509B
:019023000C40
:058EBB00900A12EFF027
:108EC000A2AF9212C2AF128DB8EF20E7F9900A124A
:098ED000E0FF1289D2A21292AF58
:018ED9002276
:108DB800A2AF9213C2AF75A0FFC2B6D2B5D2B77F29
:108DC80014DFFEAEA0C2B77F14DFFEA21392AFAFCE
:018DD8000694
:018DD9002277
:059100007F01028EBB9F
:1089D200A2AF9214C2AF8FA07F147E00EF1F70016E
:1089E2001EEF4E70F7C2B6C2B5D2B77E007F14EF4B
:1089F2001F70011EEF4E70F7C2B77E007F14EF1F8B
:0B8A020070011EEF4E70F7A21492AF3F
:018A0D002246
:108C5E00A2AF9215C2AF8FA0C2B5D2B7D2B67F1453
:108C6E007E00EF1F70011EEF4E70F7C2B77E007FC1
:0E8C7E0014EF1F70011EEF4E70F7A21592AF9B
:018C8C0022C5
:0C500C00900A13E05FF04DFFF0028EBB35
:028F7A00AD0741
:108F7C00A2AF9216C2AF128DB8EF20E7F9AF05126F
:068F8C008C5EA21692AFFC
:018F920022BC
:088A0E00E0FBA3E0FAA3E0F98C
:108A16009009F8EBF0A3EAF0A3E9F09009F8E0FB7F
:108A2600A3E0FAA3E0F9124CE560179009F8A3E475
:108A360075F001124DFEA9F0FA124CE5FF128F7A7D
:038A460080D922B2
:0B8A49009009D3EBF0A3EAF0A3E9F0E2
:108A5400A2AF9217C2AF129100E4FDFF128FC29031
:108A640009D3128A0EE4FD7F01128FC29009D61237
:0D8A74008A0E7D117F01128FC2A21792AFF2
:018A810022D2
:108FC200A2AF9218C2AFEF75F040A42D2480FF1219
:068FD2008EBBA21892AF55
:018FD8002276
:10902400AE84E4F584EF90879B93F5D3AF068F84E9
:019034002219
:10669000000000010003000500070008000A000CCC
:1066A000000E000F00110013001500160018001A4C
:1066B000001C001D001F00210023002400260028CC
:1066C000002A002B002D002F00310032003400364C
:1066D00000380039003B003D003F004000420044CC
:1066E000004600470049004B004D004E005000524C
:1066F0000054005500570059005B005C005E0060CC
:1067000000620063006500670069006A006C006E4B
:10671000007000710073007500770078007A007CCB
:10672000007E007F00810083008500860088008A4B
:10673000008C008D008F00910093009400960098CB
:10674000009A009B009D009F00A100A200A400A64B
:1067500000A800A900AB00AD00AF00B000B200B4CB
:1067600000B600B700B900BB00BD00BE00C000C24B
:1067700000C400C500C700C900CB00CC00CE00D0CB
:1067800000D200D300D500D700D900DA00DC00DE4B
:1067900000E000E100E300E500E700E800EA00ECCB
:1067A00000EE00EF00F100F300F500F600F800FA4B
:1067B00000FC00FD00FF0000000A0014001F00297B
:1067C0000033003E00480052005D00670071007C0D
:1067D00000860090009A00A500AF00BA00C400CE69
:1067E00000D900E300ED00F80102010C01160121BF
:1067F000012B01350140014A0155015F0169017416
:10680000017E01880193019D01A701B201BC01C66F
:1068100001D101DB01E501F001FA0204020E0219C7
:106820000223022D02380242024C02570261026B1F
:1068300002760280028A0295029F02AA02B402BE78
:1068400002C902D302DD02E802F202FC03070311CF
:10685000031B03260330033A0345034F0359036424
:10686000036E03780383038D039703A203AC03B67F
:1068700003C103CB03D503E003EA03F403FF0000E5
:10688000009A00F401340165018E01B001CE01E8E7
:1068900001FF02150228023A024A025A02680275F2
:1068A0000282028E029902A402AF02B902C202CB96
:1068B00002D402DC02E402EC02F402FB030203094C
:1068C000030F0316031C03220328032E033403398A
:1068D000033E03440349034E03530357035C036120
:1068E0000365036A036E03720376037A037E0382F1
:1068F0000386038A038E039103950399039C03A0E7
:1069000003A303A603AA03AD03B003B303B603B9FD
:1069100003BC03BF03C203C503C803CB03CE03D02C
:1069200003D303D603D903DB03DE03E003E303E56C
:1069300003E803EA03ED03EF03F203F403F603F9BC
:1069400003FB03FD03FF5051525456585B5F6368CD
:106950006E757D8793A2B3C8E1FF505255595E66AC
:10696000707E91ABCEFF505154575B60666F7A8951
:106970009CB5D5FF40002000155510000CCC0AAA8C
:1069800009240800071C0666055504920400038EBE
:106990000333028F022201D40199016C01470111D6
:1069A00000EA00CC00B600A3008800750066005B1A
:1069B000005100410036002E002800240020001B5A
:1069C00000170014001200100000000C0018002432
:1069D0000030003C004800540060006C00780084E7
:1069E0000090009C00A800B400C000CC00D800E4D7
:1069F00000F000FC010801140120012C01380144C1
:106A00000150015D016901750181018D019901A5A7
:106A100001B101BD01C901D501E101ED01F9020595
:106A20000211021D022902350241024D025902657E
:106A30000271027D0289029502A102AE02BA02C66B
:106A400002D202DE02EA02F60302030E031A032652
:106A50000332033E034A03560362036E037A03863E
:106A60000392039E03AA03B603C203CE03DA03E62E
:046A700003F203FF2B
:108A8200E4FFEF75F008A42434F582E43404F5839E
:108A9200E4F0A3F0FEEF75F008A42436F582E43486
:108AA20004F58375F002EE124F56E4F0A3F00EEED9
:088AB200B403E20FEFB410CA97
:018ABA002299
:0690EE001262210270D69F
:106221009004347420F090043C7410F09004447491
:1062310080F090044C7470F09004547440F0900419
:106241005C7430F09004647460F090046C7450F0ED
:10625100900699E075F01DA424B1F582E43405F5AA
:1062610083C083C0829005AEE0D082D08375F009EF
:10627100124F56E0FFC394144005EF9428400BEFF2
:10628100C3943C407AEF94505075900699E075F0B4
:106291001DA424B1F582E43405F583C083C0829046
:1062A10005AEE0D082D083129035C374139FFFE412
:1062B1009400FE74462FF58274693EF583E493756C
:1062C100F010A4FF900434E045F0F0A3E04FF0900B
:1062D1000699E075F01DA424B1F582E43405F58337
:1062E100C083C0829005AEE0D082D083129035EF9A
:1062F1009069469375F010A4FF90043C026372907C
:106301000699E075F01DA424B1F582E43405F58306
:10631100C083C0829005AEE0D082D083129035C395
:1063210074139FFFE49400FE74462FF58274693E56
:10633100F583E49375F010A4FF90043CE045F0F080
:10634100A3E04FF0900699E075F01DA424B1F58209
:10635100E43405F583C083C0829005AEE0D082D0DD
:1063610083129035EF9069469375F010A4FF900465
:1063710034E045F0F0A3E04FF0900699E075F01D90
:10638100A424B0F582E43405F583C083C08290056E
:10639100AEE0D082D08375F009124F56E0FFC3946E
:1063A100144005EF9428400BEFC3943C4042EF9416
:1063B10050503DEF75F01484ADF0EDFFC374139FA1
:1063C100FFE49400FE74462FF58274693EF583E480
:1063D1009375F010A4FF900444E045F0F0A3E04F62
:1063E100F0ED9069469375F010A4FF90044C805E27
:1063F100900699E075F01DA424B0F582E43405F50A
:1064010083C083C0829005AEE0D082D08375F0094D
:10641100124F56E075F01484ADF0EDFFC374139F75
:10642100FFE49400FE74462FF58274693EF583E41F
:106431009375F010A4FF90044CE045F0F0A3E04FF9
:10644100F0ED9069469375F010A4FF900444E04587
:10645100F0F0A3E04FF0900699E075F01DA424B28E
:10646100F582E43405F583C083C0829005AEE0D0A7
:1064710082D08375F009124F56E0FFC39414400592
:10648100EF9428400BEFC3943C4042EF9450503DB1
:10649100EF75F01484ADF0EDFFC374139FFFE49426
:1064A10000FE74462FF58274693EF583E49375F01E
:1064B10010A4FF900454E045F0F0A3E04FF0ED90FC
:1064C10069469375F010A4FF90045C805E90069974
:1064D100E075F01DA424B2F582E43405F583C08390
:1064E100C0829005AEE0D082D08375F009124F567C
:1064F100E075F01484ADF0EDFFC374139FFFE494D5
:1065010000FE74462FF58274693EF583E49375F0BD
:1065110010A4FF90045CE045F0F0A3E04FF0ED9093
:1065210069469375F010A4FF900454E045F0F0A380
:10653100E04FF0900699E075F01DA424AFF582E4D8
:106541003405F583C083C0829005AEE0D082D0834C
:1065510075F009124F56E0FFC3940C4005EF9418F3
:106561004016EFC394244005EF9430400BEFC394E1
:106571003C4043EF9448503EEF75F00C84ADF0ED94
:10658100FFC3740B9FFFE49400FE745A2FF58274CD
:10659100693EF583E49375F010A4FF900464E0452F
:1065A100F0F0A3E04FF0ED90695A9375F010A4FF5D
:1065B10090046C026687900699E075F01DA424AFE3
:1065C100F582E43405F583C083C0829005AEE0FF17
:1065D100D082D08375F009124F56E0C394489006DB
:1065E10099E075F01D4048A424AFF582E43405F527
:1065F1008375F009EF124F56E0FD90691E9375F017
:1066010010A4FF900464E045F0F0A3E04FF0EDFF2B
:10661100C374559FFFE49400FE74662FF58274697C
:106621003EF583E49375F010A4FF90046C8057A4A9
:1066310024AFF582E43405F583C083C0829005AEB2
:10664100E0D082D08375F009124F56E075F00C84CA
:10665100ADF0EDFFC3740B9FFFE49400FE745A2F5D
:10666100F58274693EF583E49375F010A4FF9004FC
:106671006CE045F0F0A3E04FF0ED90695A9375F0AE
:0F66810010A4FF900464E045F0F0A3E04FF02276
:047DB300E4FFC2FA2D
:107DB700900A03E4F0A3740AF0900A0374FFF5F045
:0E7DC700124DFEFCD3E5F09400EC940050EB5E
:107DD500E59A20E7FBEF75F008A42434F582E43436
:107DE50004F583E0F59B30FFFDC2FFE59A20E7FB34
:107DF500EF75F008A42435F582E43404F583E0F545
:107E05009B30FFFDC2FFE4FEE59A20E7FBEF75F02E
:107E150008A42436F582E43404F58375F002EE12E5
:107E25004F56E0F59B30FFFDC2FFE59A20E7FBEFDB
:107E350075F008A42437F582E43404F58375F0025F
:107E4500EE124F56E0F59B30FFFDC2FF0EEEB40378
:037E5500B7D2FAA7
:107E5800900A03E4F0A3740AF0900A0374FFF5F0A3
:0E7E6800124DFEFCD3E5F09400EC940050EBBC
:097E76000FEF64106003027DB5FA
:017E7F0022E0
:1070D600E4900A14F0900A14E0FFC39403400302FC
:1070E600734D90069EE0600F9005AEE0FEC37402FD
:1070F6009E6F60030272DF900A14E0FF25E02436DB
:10710600F582E43404F5837410F0EF25E02436F5B7
:1071160082E43404F583C083C082E0FCA3E0FDC3AF
:1071260074029F75F008A4241CF582E43404F583E8
:10713600E0FEA3E0FFD394FFEE9403400A7A0F7BB0
:10714600FC7E0F7FFC800BEF7802C333CE33CED8A4
:10715600F9FFEC4EFEED4FFFD082D083EEF0A3EFA9
:10716600F0900A14E0FF25E0243EF582E43404F5AD
:10717600837420F0EF25E0243EF582E43404F583A1
:10718600C083C082E0FCA3E0FDC374029FFFE494C9
:1071960000FE90041E75F008EF124F56EE75F008CB
:1071A600A42583F583E0FEA3E0FFD394FFEE9403CA
:1071B600400A7A007B007E007F008014C374FF9F24
:1071C600FF74039EFEEF7802C333CE33CED8F9FFA9
:1071D600EC4EFEED4FFFD082D083EEF0A3EFF090A1
:1071E6000A14E0FF25E02446F582E43404F58374AE
:1071F60030F0EF25E02446F582E43404F583C083BD
:10720600C082E0FCA3E0FDC374029FFFE49400FE8D
:1072160090042075F008EF124F56EE75F008A4257D
:1072260083F583E0FEA3E0FFD394FFEE9403400AC8
:107236007A007B007E007F008014C374FF9FFF747A
:10724600039EFEEF7802C333CE33CED8F9FFEC4E61
:10725600FEED4FFFD082D083EEF0A3EFF0900A143C
:10726600E0FF25E0244EF582E43404F5837440F013
:10727600EF25E0244EF582E43404F583C083C08212
:10728600E0FCA3E0FDC374029FFFE49400FE9004BB
:107296002275F008EF124F56EE75F008A42583F517
:1072A60083E0FEA3E0FFD394FFEE940340067E0046
:1072B6007F008014C374FF9FFF74039EFEEF780265
:1072C600C333CE33CED8F9FFEC4EFEED4FFFD0825E
:1072D600D083EEF0A3EFF08065900A14E0FF25E07E
:1072E6002436F582E43404F5837410F0EF25E024A7
:1072F6003EF582E43404F5837420F0EF25E0243E65
:10730600F582E43404F583C083C082E0440FFFA312
:10731600E044FCD082D083CFF0A3EFF0900A14E0D3
:10732600FF25E02446F582E43404F5837430F0EF5B
:1073360025E0244EF582E43404F5837440F0900A87
:0773460014E004F00270DB0B
:01734D00221D
:0890350075F009124F56E0FF2F
:07903D00EF75F01484AFF0A1
:019044002209
:087CCB00900973EEF0A3EFF045
:107CD300A984900973E0FEA3E0FFC3ED9FFFEC9E30
:107CE300900402F0A3EFF075840375C301900402BE
:107CF300E0FCA3E0FDECFF3395E08FC2EDF5C1EAB4
:107D0300FF3395E08F92EBF59190040AE004F0E0E5
:107D130004F0900404124F2500000000900404E5D1
:107D230096F0A3E595F0A3E594F0A3E593F0900412
:107D330004E0FCA3E0FDA3E0FEA3E0FF780F124EF6
:107D4300F3900404124F19900406E0FFA3E090049B
:107D530008CFF0A3EFF0AF018F84900973E0FEA387
:107D6300E0FF900409E02FF0900408E03EF0900952
:107D73007BE0FEA3E0FF900409E02FF0900408E00D
:107D83003EF0900979E0FEA3E0FF900408E0FCA335
:107D9300E0FDD39FEE6480F8EC648098400122C339
:0F7DA300EC648094805004E4FEFF22AF05AE0430
:017DB20022AE
:0690C100EF2DFFEE3CFE66
:0190C7002286
:03502D0002409AA4
:10409A00C0E0C0F0C083C082C0D075D000C000C0EC
:0D40AA0001C002C003C004C005C006C0076D
:1040B7009009F1E584F0900414E004F0758401752B
:1040C700D3FF75840275BB03C2EDD2EC30EDFD90D2
:1040D700041AE0A3F090041AE5BEF075840175D3C5
:1040E70000758402A3E0D394C0501090041AE094A2
:1040F700C040089004107401F08005900410E4F0AB
:1041070090041AE0D3948090041340057401F08062
:1041170002E4F0758400900414E0C3940C500B90F3
:104127000410E064016003024BC9900414E4F090AA
:104137000698E07003024A20900697E07003024257
:014147002E49
:104148007F07128D2B9004B8EEF0A3EFF090040BCC
:104158007401F0A374FFF0FD7C01124D9390069B4F
:10416800EFF0D3940740037407F090069BE0FE1429
:10417800900419F090040DE0FFEE6F600A90069B22
:10418800E090040DF080229004B8E0FEC3EE9401A4
:104198005009C390040EE09401500EC3EE94014000
:1041A8000E90040EE0940150069005AD7401F09055
:1041B800040BE0FCA3E0FD9004B8E0FEA3E0FF12CE
:1041C8004D93AE04AF05E4FCFD9005A8124F19907D
:1041D80005A8E0FCA3E0FDA3E0FEA3E0FF780F1232
:1041E8004F069005A8124F199005A8E0FCA3E0FD22
:1041F800A3E0FEA3E0FFC006C00790040BE0FEA307
:10420800E0FBAA06E4F9F8D007D006124E50900554
:10421800A8124F199004B8E0FFA3E090040ECFF065
:03422800A3EFF011
:10422B000243D090069BE075F01DA424CBF582E4ED
:10423B003405F583E0FF900412F09004117401F043
:10424B00BF010B900413E06005900411E4F090049F
:10425B0012E0FFB40208A3E07004900411F0EF64C5
:10426B00036007900412E0B40408900410E070029D
:0B427B00A3F0900411E070030243D098
:104286007F07128D2B9009F3EEF0A3EFF090069BBB
:10429600E075F01DA424CAF582E43405F583E02513
:1042A600E02474F582E43469F583E493FE740193A3
:1042B600FFE4FCFD900415124F19900415E0FCA3D1
:1042C600E0FDA3E0FEA3E0FFC004C005C006C007F2
:1042D6009009F3E0FEA3E0FF7C007D09124D81EE1C
:1042E600C4540F2401FFE433AB07FAE4F9F8D0070E
:1042F600D006D005D004124E50900415124F19E482
:10430600FFFEFDFC900415E0F8A3E0F9A3E0FAA394
:10431600E0FBC3124EE2700A900415124F2500000E
:1043260000019005A8E0FCA3E0FDA3E0FEA3E0FFEA
:10433600900415E0F8A3E0F9A3E0FAA3E0FBEF2B65
:10434600FFEE3AFEED39FDEC38FC9005A8124F1948
:10435600E47FFF7E7FFDFC9005A8E0F8A3E0F9A3CB
:10436600E0FAA3E0FBD3124EE2502190069BE075E3
:10437600F01DA424CBF582E43405F583E0FF640345
:104386006004EFB4042B900410E0602590069BE0D7
:1043960004F090069AE0FF90069BE0D39F4002E46B
:1043A600F09005A8124F25000000009005AD74019D
:1043B600F090069BE014FF90069AE0FEEFD39E4035
:0A43C60004AF068000900419EFF028
:1043D0009009F2E4F09009F2E0FFC3940340030275
:1043E0004BC090069BE0FE75F01DA424B6F582E458
:1043F0003405F58375F009EF124F56E07016EE752F
:10440000F01DA424CBF582E43405F583E064036059
:10441000030244B7900419E075F01DA424AFF5829F
:10442000E43405F583C083C0829009F2E0FDD082B8
:10443000D08375F009124F56E025E024C8F582E4D8
:104440003469F583E493FE740193FFC006C00790BE
:10445000069BE075F01DA424AFF582E43405F583D6
:1044600075F009ED124F56E025E024C8F582E434DA
:1044700069F583E493FE740193FFFDAC06C006C0AA
:10448000079009F2E075F003A4247EF582E4340974
:10449000F583E0FF128AF490097BEEF0A3EFF09031
:1044A00009797403F0A374FFF0D005D004D007D0CD
:1044B00006FB7A7F024560900419E075F01DA42484
:1044C000AFF582E43405F583C083C0829009F2E041
:1044D000FDD082D08375F009124F56E025E024C844
:1044E000F582E43469F583E493FE740193FFC0061A
:1044F000C00790069BE075F01DA424AFF582E4345C
:1045000005F58375F009ED124F56E025E024C8F556
:1045100082E43469F583E493FE740193FFFDAC06F5
:10452000C006C0079009F2E075F003A4247EF5826E
:10453000E43409F583E0FF128AF490097BEEF0A3DE
:10454000EFF09005A8A3A3E0FEA3E0FBAA06900964
:10455000797403F0A374FFF0D005D004D007D0061F
:10456000127CCB9009F2E075F008A4241CF582E4DB
:104570003404F583EEF0A3EFF090069BE0FF75F0B6
:104580001DA424B7F582E43405F583C083C082906E
:1045900009F2E0D082D08375F009124F56E0701313
:1045A000EF75F01DA424CBF582E43405F583E064B7
:1045B000037078900419E075F01DA424B2F582E42C
:1045C0003405F583C083C0829009F2E0FDD082D02B
:1045D0008375F009124F56E025E024B6F582E434E5
:1045E00067F583E493FE740193FF90069BE075F0FA
:1045F0001DA424B2F582E43405F58375F009ED12AB
:104600004F56E025E024B6F582E43467F583E49361
:10461000FC740193FD9009797403F0A374FFF0A377
:10462000E4F0A3F07BFF7A7F0246B2900419E075B4
:10463000F01DA424B2F582E43405F583C083C08262
:104640009009F2E0FDD082D08375F009124F56E058
:1046500025E024B6F582E43467F583E493FE740123
:1046600093FFC006C00790069BE075F01DA424B21E
:10467000F582E43405F58375F009ED124F56E02517
:10468000E024B6F582E43467F583E493FE74019385
:10469000FDAC069005A8A3A3E0FEA3E0FBAA06904C
:1046A00009797403F0A374FFF0A3E4F0A3F0D0073A
:1046B000D006127CCB9009F2E075F008A42422F514
:1046C00082E43404F583EEF0A3EFF090069BE0FF64
:1046D00075F01DA424B4F582E43405F583C083C0CD
:1046E000829009F2E0FDD082D08375F009124F5616
:1046F000E07016EF75F01DA424CBF582E43405F5C7
:1047000083E0640360030247A0900419E075F01D84
:10471000A424B0F582E43405F58375F009ED124F59
:1047200056E025E024B6F582E43467F583E493FE91
:10473000740193FFC006C00790069BE075F01DA4AE
:1047400024B0F582E43405F58375F009ED124F5677
:10475000E025E024B6F582E43467F583E493FE7443
:104760000193FFFDAC06C006C0079009F2E075F0AA
:1047700003A42480F582E43409F583E0FF1287A3C3
:1047800090097BEEF0A3EFF09009797403F0A37425
:10479000FFF0D005D004D007D006FB7A7F0248494D
:1047A000900419E075F01DA424B0F582E43405F5F9
:1047B00083C083C0829009F2E0FDD082D08375F07F
:1047C00009124F56E025E024B6F582E43467F583FC
:1047D000E493FE740193FFC006C00790069BE0754A
:1047E000F01DA424B0F582E43405F58375F009EDDD
:1047F000124F56E025E024B6F582E43467F583E4F1
:1048000093FE740193FFFDAC06C006C0079009F249
:10481000E075F003A42480F582E43409F583E0FF19
:104820001287A390097BEEF0A3EFF09005A8A3A355
:10483000E0FEA3E0FBAA069009797403F0A374FFDD
:10484000F0D005D004D007D006127CCB9009F2E05E
:1048500075F008A4241EF582E43404F583EEF0A379
:10486000EFF090069BE0FF75F01DA424B5F582E4FF
:104870003405F583C083C0829009F2E0FDD082D078
:104880008375F009124F56E07016EF75F01DA424E1
:10489000CBF582E43405F583E06403600302494606
:1048A000900419E075F01DA424B1F582E43405F5F7
:1048B0008375F009ED124F56E025E024B6F582E449
:1048C0003467F583E493FE740193FFC006C007903C
:1048D000069BE075F01DA424B1F582E43405F58350
:1048E00075F009ED124F56E025E024B6F582E43468
:1048F00067F583E493FE740193FFFDAC06C006C028
:10490000079009F2E075F003A4247FF582E43409EE
:10491000F583E0FF128AF4C006C0077F03128AF411
:10492000D0E02FFFD0E03E90097BF0A3EFF090099C
:10493000797403F0A374FFF0D005D004D007D0063B
:10494000FB7A7F0249FE900419E075F01DA424B1A2
:10495000F582E43405F583C083C0829009F2E0FD5E
:10496000D082D08375F009124F56E025E024B6F5C9
:1049700082E43467F583E493FE740193FFC006C0BC
:104980000790069BE075F01DA424B1F582E4340580
:10499000F58375F009ED124F56E025E024B6F58257
:1049A000E43467F583E493FE740193FFFDAC06C025
:1049B00006C0079009F2E075F003A4247FF582E4B5
:1049C0003409F583E0FF128AF4C006C0077F0312A2
:1049D0008AF4D0E02FFFD0E03E90097BF0A3EFF007
:1049E0009005A8A3A3E0FEA3E0FBAA0690097974B2
:1049F00003F0A374FFF0D005D004D007D006127CDA
:104A0000CB9009F2E075F008A42420F582E4340488
:104A1000F583EEF0A3EFF09009F2E004F00243D545
:104A20009009F2E4F0900699E075F01DA424AFF52A
:104A300082E43405F583C083C0829009F2E0FDD0A2
:104A400082D08375F009124F56E025E024C8F58224
:104A5000E43469F583E493FE740193FFC006C00754
:104A6000ED75F003A4247EF582E43409F583E0FFBC
:104A7000128AF4AD07AC06D007D0061290C1900997
:104A8000F2E0FD75F008A4241CF582E43404F583FB
:104A9000EEF0A3EFF0900699E075F01DA424B2F5B6
:104AA00082E43405F58375F009ED124F56E025E0F8
:104AB00024B6F582E43467F583E493FE740193FF32
:104AC000E4FDFC1290C19009F2E0FD75F008A42409
:104AD00022F582E43404F583EEF0A3EFF09006991A
:104AE000E075F01DA424B0F582E43405F58375F07B
:104AF00009ED124F56E025E024B6F582E43467F55F
:104B000083E493FE740193FFC006C007ED75F003C4
:104B1000A42480F582E43409F583E0FF1287A3AD75
:104B200007AC06D007D0061290C19009F2E0FD75DF
:104B3000F008A4241EF582E43404F583EEF0A3EF1C
:104B4000F0900699E075F01DA424B1F582E43405D7
:104B5000F58375F009ED124F56E025E024B6F58295
:104B6000E43467F583E493FE740193FFC006C00745
:104B7000ED75F003A4247FF582E43409F583E0FFAA
:104B8000128AF4C006C0077F03128AF4D0E02FFD1A
:104B9000D0E03EFCD007D0061290C19009F2E0753B
:104BA000F008A42420F582E43404F583EEF0A3EFAA
:104BB000F09009F2E004F0E0C394035003024A25A8
:104BC000128A821290EE127DB3758401C2CF9009D1
:044BD000F1E0F58497
:104BD400D007D006D005D004D003D002D001D00035
:0B4BE400D0D0D082D083D0F0D0E032DF
:108BFF0090097E7404F090098104F090098404F0C8
:108C0F00E490097FF090098204F090098504F090B8
:108C1F0009807405F090098304F090098604F0220E
:108AF400AD84E4F5848FBBC2EDD2EC30EDFD900A79
:108B040005E5BFF0A3E5BEF0900A05E0FEA3E0781A
:108B140002CEC313CE13D8F9F0EE900A05F0AF05D8
:078B24008F84E0FEA3E0FFD7
:018B2B002227
:108D2B00AE84E4F5848FBBC2EDD2EC30EDFD900A3E
:108D3B0007E5BFF0A3E5BEF0AF068F84900A07E00E
:048D4B00FEA3E0FFA4
:018D4F002201
:1087A300AD84ACE775840253E7FBE5E85401FB8F26
:1087B300BBC2EDD2EC30EDFDE4900A09F0A3E5BEB7
:1087C300F0900A09E0FEA3E07802C333CE33CED89B
:1087D300F9F0EE900A09F053E8FEAF03EB42E8AF7D
:0C87E300048FE7AF058F84E0FEA3E0FFE9
:0187EF002267
:035009000250064C
:03500600C28B3228
:03503300028ABB33
:0D8ABB00C0E0C083C082C0D075D000C007ED
:108AC800AF8475840275BB03C2EDD2EC30EDFD9026
:108AD8000A15E5BEF0E5E830E00353E7FBC2CF8FA7
:018AE8008409
:0B8AE900D007D0D0D082D083D0E03284
:03503600029105DF
:0491050053E7F33207
:04840200410792009C
:0690F400E4900792F02257
:0790C8009007927401F022F1
:0585CE00900A0BEFF024
:1085D3001290B9E4900A0CF0900A0BE0FFA3E0FEBE
:1085E300C39F502A75F0EBEEA42401F582E5F03425
:1085F300D0AF82FE7B017A0579AF9009B8E4F0A38E
:1086030074EBF0128888900A0CE004F080CA7ED0E4
:0A8613007F007D0112812C028CE033
:10501B001290B97ED07F0090069DE0FD12812C028C
:02502B008CE017
:1087F000900A0D7402F0E4A3F01290B97EEB7F8C26
:108800007B017A0A790D9009B8E4F0A304F012888C
:10881000887EEB7F8B7B017A0A790E9009B8E4F0B1
:10882000A304F0128888128CE07E007FEB7D007B31
:0D883000017A0579AF124F8E7F1E0285CEB2
:108E5C009006A5E0700374FFF0200C13300E1090F8
:108E6C000792E070089006A3E0FF128DDAD20C2274
:03503000028E5C91
:108E7C0090EB8BE493F46007A3E493640260031219
:108E8C0087F0E49006A6F090D0009390069DF02217
:108B2C00A2AF9219C2AF9006A6E0FFC3941E5021CB
:108B3C00EF75F0EBA42401F974D035F0FA7BFF78D3
:108B4C00AF7C057D017E007FEB124CBF128995C274
:058B5C000CA21992AF0C
:018B610022F1
:108B62009006A6E0C3941E502B1290B99006A6E080
:108B720075F0EBA42401F582E5F034D0AF82FE7BE0
:108B8200017A0579AF9009B8E4F0A374EBF012888A
:058B920088128CE022B6
:0690FA00128B62C20C2281
:0790CF00300D031290FA229C
:10899500E490069AF090069AE0FFC394085021EF00
:1089A50075F01DA424CBF582E43405F583E0FF645E
:1089B50004600DEF6405600890069AE004F080D528
:0D89C50090069AE0C3940840037407F02266
:087E8000900948EDF0A3EBF0BE
:107E8800A3E004F090094DEFF0A3EBF0900948E06F
:107E9800FF90094DE0FED39F4003027F3475F0EB5D
:107EA800EEA42401F582E5F034D0AF8290094FF0BA
:107EB800A3EFF090094EE075F0EBA42401F582E5FC
:107EC800F034D0AF82900951F0A3EFF0E490094B61
:107ED800F0A3F0900951E475F001124DFEAFF0FEE9
:107EE80090094FE0FCA3E0F5828C83E493FD1281B6
:107EF8002C900950E004F0700690094FE004F090CF
:107F0800094CE004F0700690094BE004F0C39009B6
:107F18004CE094EB90094BE0940040B7128CE09051
:107F2800094DE004F0A3E004F0027E949006A6E078
:107F3800FF900949E0D39F5009A3E0C39F40031273
:027F48008B2C80
:017F4A002214
:0F734E0090095FEDF090095EEFF0900960EBF0B1
:10735D00900965EFF0A3EBF090095FE0FF900965F0
:10736D00E0D39F40030274C9A3E075F0EBA42401A0
:10737D00F582E5F034D0AF82900961F0A3EFF0E42F
:10738D00900967F0A3F0900967E0FEA3E0FFC394B6
:10739D00EBEE94005038900961E0FCA3E0F5828C8F
:1073AD0083E493FD74A72FF582E43406F583EDF0A5
:1073BD00900962E004F07006900961E004F0900914
:1073CD0068E004F070C0900967E004F080B890099F
:1073DD0065E075F0EBA42401F582E5F034D0AF82C1
:1073ED00900963F0A3EFF0900966E075F0EBA4242B
:1073FD0001F582E5F034D0AF82900961F0A3EFF092
:10740D00E4900967F0A3F0900961E475F001124D65
:10741D00FEAFF0FE900963E0FCA3E0F5828C83E4FF
:10742D0093FD12812C900964E004F07006900963BD
:10743D00E004F0900968E004F07006900967E0043C
:10744D00F0C3900968E094EB900967E0940040B7B1
:10745D00900965E075F0EBA42401F582E5F034D0D8
:10746D00AF82900963F0A3EFF0E4900967F0A3F009
:10747D00900967E0FCA3E0FDC394EBEC9400502C65
:10748D00900963E475F001124DFEAFF0FE74A72D67
:10749D00F582E43406F583E0FD12812C900968E055
:1074AD0004F070CC900967E004F080C4128CE09079
:1074BD000965E004F0A3E004F00273659006A6E010
:1074CD00FF900960E0FED39F502090095EE0FDA380
:1074DD00E0C39DFDE49400FCEE7A002DFDEA3CFC3A
:1074ED00C3ED9F7480F86C9850139006A6E0FF9042
:1074FD00095EE0D39F5009A3E0C39F4003128B2C7C
:01750D00225B
:0B7F4B00900987EFF0A3EDF0A3EBF02E
:107F5600A2AFE433A3F0C2AF1290E2900988E0FE2C
:107F6600900987E0FDEDFF90098FEEF0A3EFF0E4B6
:107F760090098BF0900989E0FF90098FE0FCA3E05F
:107F8600FD7B017A0679A79009A9E4F0A374EBF0CA
:107F9600128D96900990E024EBF090098FE0340062
:107FA600F090098BE075F0EBA42401F974D035F05C
:107FB600FAA374FFF0A3EAF0A3E9F01290B99009CE
:107FC6008CA3E0FAA3E0AE02FF7B017A0679A790C4
:107FD60009B8E4F0A374EBF0128888128CE09009DB
:107FE6008BE004F0E0C3941E408A9006A3E0FF12E3
:0A7FF600906290098AE024FF92AF28
:01800000225D
:0B80010090099AEFF0A3EDF0A3EBF064
:10800C00A2AFE433A3F0C2AF1290E290099BE0FE62
:10801C0090099AE0FDEDFF90099FEEF0A3EFF0E4DC
:10802C0090099EF090099EE0FFC3941E504C75F091
:10803C00EBEFA42401F582E5F034D0AF82FE900979
:10804C00A1F0FAA3EFF0FB90099CE0FF90099FE0F0
:10805C00FCA3E0FDA9037BFF9009B1E4F0A374EB52
:10806C00F0128F2E9009A0E024EBF090099FE034E1
:10807C0000F090099EE004F080AA9006A3E0FF12A5
:0A808C00906290099DE024FF92AF7E
:0180960022C7
:03000000024000BB
:03000300025003A5
:03000B000250069A
:030013000250098F
:03001B0002500C84
:0300230002500F79
:03002B000250126E
:0300330002501563
:03003B0002501858
:0300430002501B4D
:03004B0002501E42
:0300530002502137
:03005B000250242C
:0300630002502721
:03006B0002502A16
:0300730002502D0B
:03007B0002503000
:03008300025033F5
:03008B00025036EA
:03009300025039DF
:03009B0002503CD4
:0300A30002503FC9
:10400000787FE4F6D8FD9000007F007E20E4F0A3E6
:0A401000DFFCDEFA75812302405543
:10401A00025039E493A3F8E493A34003F68001F233
:10402A0008DFF48029E493A3F85407240CC8C333A7
:10403A00C4540F4420C8834004F456800146F6DF76
:10404A00E4800B010204081020408090839FE47EE4
:10405A00019360BCA3FF543F30E509541FFEE4936B
:10406A00A360010ECF54C025E060A840B8E493A332
:10407A00FAE493A3F8E493A3C8C582C8CAC583CA5D
:10408A00F0A3C8C582C8CAC583CADFE9DEE780BE15
:018406000075
:104BEF00E709F608DFFA8046E709F208DFFA803EA8
:104BFF0088828C83E709F0A3DFFA8032E309F60895
:104C0F00DFFA8078E309F208DFFA807088828C83FC
:104C1F00E309F0A3DFFA806489828A83E0A3F608B0
:104C2F00DFFA805889828A83E0A3F208DFFA804C8A
:104C3F0080D280FA80C680D4806980F28033801061
:104C4F0080A680EA809A80A880DA80E280CA8033CA
:104C5F0089828A83ECFAE493A3C8C582C8CCC58342
:104C6F00CCF0A3C8C582C8CCC583CCDFE9DEE78012
:104C7F000D89828A83E493A3F608DFF9ECFAA9F091
:104C8F00EDFB2289828A83ECFAE0A3C8C582C8CCE7
:104C9F00C583CCF0A3C8C582C8CCC583CCDFEADE00
:104CAF00E880DB89828A83E493A3F208DFF980CC62
:104CBF0088F0EF60010E4E60C388F0ED2402B4045B
:104CCF000050B9F582EB2402B4040050AF23234502
:064CDF008223904C3F739C
:104CE500BB010689828A83E0225002E722BBFE02CD
:094CF500E32289828A83E4932200
:104CFE00BB010CE58229F582E5833AF583E022506B
:104D0E0006E92582F8E622BBFE06E92582F8E222B4
:0D4D1E00E58229F582E5833AF583E49322CE
:104D2B00BB010989828A83F8E028F022500327F718
:104D3B0022BBFE05F8E328F3228A838982F8E493E9
:024D4B0028221C
:104D4D00BB010689828A83F0225002F722BBFE0145
:024D5D00F3223F
:104D5F00F8BB010DE58229F582E5833AF583E8F08A
:104D6F00225006E92582C8F622BBFE05E92582C836
:024D7F00F2221E
:104D8100EF8DF0A4A8F0CF8CF0A428CE8DF0A42E46
:024D9100FE2200
:104D9300BC000BBE0029EF8DF084FFADF022E4CC04
:104DA300F875F008EF2FFFEE33FEEC33FCEE9DECCD
:104DB300984005FCEE9DFE0FD5F0E9E4CEFD22ED13
:104DC300F8F5F0EE8420D21CFEADF075F008EF2F5D
:104DD300FFED33FD4007985006D5F0F222C398FD4E
:054DE3000FD5F0EA22EB
:104DE800C5F0F8A3E028F0C5F0F8E5821582700256
:064DF8001583E038F022F3
:104DFE00A3F8E0C5F025F0F0E58215827002158368
:064E0E00E0C838F0E822C4
:104E140075F008758200EF2FFFEE33FECD33CDCC55
:104E240033CCC58233C5829BED9AEC99E5829840D8
:104E34000CF582EE9BFEED9AFDEC99FC0FD5F0D6B5
:104E4400E4CEFBE4CDFAE4CCF9A88222B800C1B9DF
:104E54000059BA002DEC8BF084CFCECDFCE5F0CB1D
:104E6400F97818EF2FFFEE33FEED33FDEC33FCEB56
:104E740033FB10D703994004EB99FB0FD8E5E4F911
:104E8400FA227818EF2FFFEE33FEED33FDEC33FCFE
:104E9400C933C910D7059BE99A4007EC9BFCE99AF2
:104EA400F90FD8E0E4C9FAE4CCFB2275F010EF2F37
:104EB400FFEE33FEED33FDCC33CCC833C810D70737
:104EC4009BEC9AE899400AED9BFDEC9AFCE899F872
:0E4ED4000FD5F0DAE4CDFBE4CCFAE4C8F92205
:104EE200EB9FF5F0EA9E42F0E99D42F0E89C45F026
:014EF200229D
:104EF300E8600FECC313FCED13FDEE13FEEF13FF9D
:034F0300D8F122C0
:104F0600E8600FEFC333FFEE33FEED33FDEC33FC09
:034F1600D8F122AD
:0C4F1900ECF0A3EDF0A3EEF0A3EFF0220B
:104F2500A8828583F0D083D082124F3C124F3C1269
:104F35004F3C124F3CE473E493A3C583C5F0C5838E
:104F4500C8C582C8F0A3C583C5F0C583C8C582C8D6
:014F55002239
:0C4F5600A42582F582E5F03583F5832266
:104F6200D083D082F8E4937012740193700DA3A3DE
:104F720093F8740193F5828883E4737402936860F2
:064F8200EFA3A3A380DFF2
:064F88008A838982E473B4
:106A7400E50D24FDF582E43408F583E0050D22904C
:106A840008FA3007039008FDE475F001124FBA02CA
:106A94004CE52000E97F2ED2008018EF540F24909B
:106AA400D43440D4FF30040BEF24BFB41A00500395
:106AB4002461FFE50E6002150E0511E51170020553
:106AC4001030070E9008FAE475F001124FBAEF0285
:106AD4004D4D028CB97403D2078003E4C207F50D4F
:106AE4009008FA124FD1E4F50EF510F511E50E6099
:106AF400077F20126AB780F5750FFFC201C200C27A
:106B040002C203C205C206C208126A83FF700D30B6
:106B140007057F00126AC8AF11AE1022B4255FC208
:106B2400D5C204126A83FF24D0B40A00501A75F047
:106B34000A780E30D50508B6FF0106C6A426F6204D
:106B4400D5047002D20380D924CFB41A00EF5004C4
:106B5400C2E5D204026CC9D20180C6D20080C0D280
:106B64000280BCD2D580BAD20580B47F20126AB725
:106B74002002077401B50E0040F1126A74FF126A14
:106B8400B7026AF1D208D2068095126A74FB126ABF
:106B940074FA126A74F94A4B7006799A7A6D7BFF1B
:106BA40020022EE50E602A7E008E82758300124C30
:106BB400FE60060EEE650F70F0C2D5EBC0E0EAC0D1
:106BC400E0E9C0E0EE126D10D0E0F9D0E0FAD0E0D8
:106BD400FB124CE5FF60AAEBC0E0EAC0E0E9C0E0CC
:106BE400126AB7D0E02401F9D0E03400FAD0E0FB17
:106BF400E50F0460DCD50FD980877BFF7A6D790CB3
:106C0400D202809C791080027908C206C2088008EA
:106C1400D2D5790A8004790AC2D5E50F047002F549
:106C24000FE4FAFDFEFF126A74FC7B0820011312C4
:106C34006A74FD7B1030000A126A74FE126A74FFD3
:106C44007B20EC3382D592D55013C3E43000069FE9
:106C5400FFE49EFEE42001039DFDE49CFCE4CBF8EC
:106C6400C201EC700CCFCECDCCE824F8F870F380E0
:106C740017C3EF33FFEE33FEED33FDEC33FCEB33A0
:106C8400FB994002FB0FD8E9EB300105F8D0E0C4D2
:106C940048B201C0E00AEC4D4E4F78207B0070C230
:106CA400EAB50F0040BCC0E0126D12D0F0D0E02075
:106CB4000104C4C0E0C4B201C0F0126AA0D0F0D58F
:106CC400F0EB026AF1124F626B8E536C08586B5FE3
:106CD4004C6B5B426C0C4F6C14446C14496B7443E6
:086CE4006C1A556BFE466BFEB5
:106CEC00456BFE476DBA506B632D6B672E6B8A2B11
:106CFC006B6B236B88206DA32A6B234800006B827F
:106D0C003F3F3F00790AA2D5200314300509B91082
:106D1C00020404B9080104A2D52006025001042083
:106D2C0002689202B50E005034C0E07F2030031987
:106D3C007F30A20272067205500F126D69C202C238
:106D4C0006C205C2087F30800F300503E9C0E0128F
:106D5C006AB7300503D0E0F9D0E0B50ECC3005179A
:106D6C007F30B9100C126AB77F583004077F7880D7
:106D7C0003B90803126AB73002057F2D026AB77F88
:106D8C00202008F87F2B2006F322920280CF286E59
:106D9C00756C6C2900D201126A743001F8C201784A
:106DAC000E30D50108F6026B232D50434958126A58
:106DBC00742403B405004001E4906DB593126AA8E5
:0D6DCC00743A126AA8D203750E04026C0816
:104F8E00EF4E6012EF60010EEDBB010B89828A833A
:104F9E00F0A3DFFCDEFA2289F05007F709DFFCA947
:0C4FAE00F022BBFEFCF309DFFCA9F0229E
:104FBA00F8E0FBA3A3E0F925F0F0E5821582700280
:074FCA001583E0FA38F02224
:094FD100EBF0A3EAF0A3E9F022E1
:108CB900EFB40A07740D128CC4740A309811A8997C
:108CC900B8130CC2983098FDA899C298B811F6301B
:078CD90099FDC299F59922F3
:00000001FF
